:1000000019C033C032C031C030C02FC02EC02DC087
:100010002CC02BC02AC029C028C027C026C025C09C
:1000200024C023C022C021C020C01FC01EC01DC0CC
:100030001CC01BC011241FBECFEFD2E0DEBFCDBF5E
:1000400011E0A0E0B1E0EAE3F1E002C005900D921A
:10005000A031B107D9F711E0A0E1B1E001C01D92D4
:10006000A131B107E1F73FD066C0CACF809110013E
:1000700090E0FC01E050FF4F208125B9FC01ED5FCD
:10008000FE4F20812BB9875F9E4FFC0180818093BA
:100090007C00089508951F920F920FB60F921124BD
:1000A0002F933F934F935F936F937F938F939F9380
:1000B000AF93BF93EF93FF93809110018F5F809375
:1000C0001001D4DFFF91EF91BF91AF919F918F917C
:1000D0007F916F915F914F913F912F910F900FBE44
:1000E0000F901F90189584B1896384B98FE38AB902
:1000F0008AB18F738AB98BB18F738BB9F894809161
:100100007B00806480937B0080917A008F7780935E
:100110007A0080B7826080BF80B7886080BF80919E
:10012000010185B9809104018BB980910A01809306
:0A0130007C007894FFCFF894FFCF15
:10013A0009112112062421091802010302010300F0
:00000001FF
